:020000040000FA
:2B000000FFFF62FF2500FFFFFFFFFFFFFFFFFFFFFFFFFFFFFFFFFFFFFFFFFFFFFFFFFFFFFFFFFFFFFFFFFFFFFFFFFF76
:2B002B00601886611886611886611986611886611886010000000018866119866118866118866118866118866180E64E
:2B005600401004411004411004E1100441100441100401000000001004E110044110044110044110044110044100C57E
:2B008100000000000000000000000000000000000000000000000000000000000000000000000000000000000080E7ED
:2B00AC00000000000000000000000000000000000000000000000000000000000000000000000000000000000080E7C2
:2B00D700000000000000000000800000000000000000000000000000008400000000000000000000000000000000A357
:2B010200000000000000000000800000000000000000000000000000002000000000000000000000000000000000ED45
:2B012D00000000000000000000000000000000000000000000000000000000000000000000000000000000000080E740
:2B015800000000000000000000000000000000000000000000000000000000000000000000000000000000000080E715
:2B018300000000000000000000000000000000000000000000000000000000000000000000000000000000000080E7EA
:2B01AE00000000000000000000000000000000000000000000000000000000000000000000000000000000000080E7BF
:2B01D900000000000000000000000000000000000000000000000000000000000000000000000000000000000080E794
:2B020400000000000000000000000000000000000000000000000000000000000000000000000000000000000080E768
:2B022F00000000000000000000000000000000000000000000000000000000000000000000000000000000000080E73D
:2B025A000000000000000000000000000000000000000000000000000000000000000000000000000000000000A0C514
:2B028500000000000000000000000000000000000000000000000000000000000000000000000000000000000080E7E7
:2B02B0000000000000000000000000000000000000000000000000000000000000000000000000000000000000A0C5BE
:2B02DB00000000000000000000000000000000000000000000000000000000000000000000000000000000000080E791
:2B030600000000000000000000000000000000000000000000000000000000000000000000000000000000000080E765
:2B033100000000000000000000000000000000000000000000000000000000000000000000000000000000000080E73A
:2B035C00000000000000000000000000000000000000000000000000000000000000000000000000000000000080E70F
:2B038700000000000000000000000000000000000000000000000000020000000000000000000000000000000080E5E4
:2B03B200020000000000000000000000000000000000000000000000020000000000000000000000000000000008EF25
:2B03DD00000000000000000000000000000000000000000000000000000000000000000000000000000000000080E78E
:2B040800000000000000000000000000000000000000000000000000000000000000000000000000000000000080E762
:2B043300000000000000000000000000000000000000000000000000000000000000000000000000000000000080E737
:2B045E00000000000000000000000000000000000000000000000000000000000000000000000000000000000080E70C
:2B048900020000000000000000000000000000000000000000000000000000000000000000000000000000000008ED51
:2B04B400800008800008800008800008800008800008000000000020000220000220000220000220000220000280E7BA
:2B04DF00800008800008800008800008800008800008000000000020000220000220000220000220000220000280E78F
:2B050A00000000000000000000000000000000000000000000000000000000000000000000000000000000000080E75F
:2B053500020000000000000000000000000000000000000000000000000000000000000000000000000000000008EDA4
:2B056000000000000000000000000000000000000000000000000000000000000000000000000000000000000008EF79
:2B058B00000000000000000000000000000000000000000000000000000000000000000000000000000000000090F6BF
:2B05B600000000000000000000000000000000000000000000000000000000000000000000000000000000000008EF23
:2B05E100000000000000000000000000000000000000000000000000000000000000000000000000000000000008EFF8
:2B060C00020000000000000000000000000000000000000000000000000000000000000000000000000000000008EDCC
:2B063700000000000000000000000000000000000000000000000000000000000000000000000000000000000080E731
:2B066200000000000000000000000000000000000000000000000000000000000000000000000000000000000080E706
:2B068D00000000000000000000000000000000000000000000000000000000000000000000000000000000000080E7DB
:2B06B800020000000000000000000000000000000000000000000000000000000000000000000000000000000008ED20
:2B06E300000000000000000000000000000000000000000000000000000000000000000000000000000000000080E785
:2B070E00000000000000000000000000000000000000000000000000000000000000000000000000000000000080E759
:2B073900000000000000000000000000000000000000000000000000000000000000000000000000000000000080E72E
:2B076400000000000000000000000000000000000000000000000000000000000000000000000000000000000080E703
:2B078F00020000000000000000000000000000000000000000000000000000000000000000000000000000000008ED48
:2B07BA00000000000000000000000000000000000000000000000000000000000000000000000000000000000080E7AD
:2B07E500000000000000000000000000000000000000000000000000000000000000000000000000000000000080E782
:2B081000000000000000000000000000000000000000000000000000000000000000000000000000000000000080E756
:2B083B00020000000000000000000000000000000000000000000000000000000000000000000000000000000008ED9B
:2B086600000000000000000000000000000000000000000000000000000000000000000000000000000000000080E700
:2B089100000000000000000000000000000000000000000000000000000000000000000000000000000000000080E7D5
:2B08BC00000000000000000000000000000000000000000000000000000000000000000000000000000000000080E7AA
:2B08E700000000000000000000000000000000000000000000000000000000000000000000000000000000000080E77F
:2B091200020000000000000000000000000000000000000000000000000000000000000000000000000000000008EDC3
:2B093D00000000000000000000000000000000000000000000000000000000000000000000000000000000000080E728
:2B096800000000000000000000000000000000000000000000000000000000000000000000000000000000000080E7FD
:2B099300000000000000000000000000000000000000000000000000000000000000000000000000000000000080E7D2
:2B09BE00020000000000000000000000000000000000000000000000000000000000000000000000000000000008ED17
:2B09E900000000000000000000000000000000000000000000000000000000000000000000000000000000000080E77C
:2B0A1400000000000000000000000000000000000000000000000000000000000000000000000000000000000080E750
:2B0A3F00000000000000000000000000000000000000000000000000000000000000000000000000000000000080E725
:2B0A6A00000000000000000000000000000000000000000000000000000000000000000000000000000000000080E7FA
:2B0A9500020000000000000000000000000000000000000000000000000000000000000000000000000000000008ED3F
:2B0AC000000000000000000000000000000000000000000000000000000000000000000000000000000000000080E7A4
:2B0AEB00000000000000000000000000000000000000000000000000000000000000000000000000000000000080E779
:2B0B1600000000000000000000000000000000000000000000000000000000000000000000000000000000000080E74D
:2B0B4100020000000000000000000000000000000000000000000000000000000000000000000000000000000008ED92
:2B0B6C00020000000000000000000000000000000000000000000000000000000000000000000000000000000008ED67
:2B0B9700040000000000000000000000000000000000000000000000000000000000000000000000000000000090F2AD
:2B0BC200020000000000000000000000000000000000000000000000000000000000000000000000000000000008ED11
:2B0BED00020000000000000000000000000000000000000000000000000000000000000000000000000000000008EDE6
:2B0C1800020000000000000000000000000000000000000000000000000000000000000000000000000000000008EDBA
:2B0C4300000000000000000000000000000000000000000000000000000000000000000000000000000000000080E71F
:2B0C6E00000000000000000000000000000000000000000000000000000000000000000000000000000000000080E7F4
:2B0C9900000000000000000000000000000000000000000000000000000000000000000000000000000000000080E7C9
:2B0CC400020000000000000000000000000000000000000000000000000000000000000000000000000000000008ED0E
:2B0CEF00000000000000000000000000000000000000000000000000000000000000000000000000000000000080E773
:2B0D1A00000000000000000000000000000000000000000000000000000000000000000000000000000000000080E747
:2B0D4500000000000000000000000000000000000000000000000000000000000000000000000000000000000080E71C
:2B0D7000000000000000000000000000000000000000000000000000000000000000000000000000000000000080E7F1
:2B0D9B00020000000000000000000000000000000000000000000000000000000000000000000000000000000008ED36
:2B0DC600000000000000000000000000000000000000000000000000000000000000000000000000000000000080E79B
:2B0DF100000000000000000000000000000000000000000000000000000000000000000000000000000000000080E770
:2B0E1C00000000000000000000000000000000000000000000000000000000000000000000000000000000000080E744
:2B0E4700020000000000000000000000000000000000000000000000000000000000000000000000000000000008ED89
:2B0E7200000000000000000000000000000000000000000000000000000000000000000000000000000000000080E7EE
:2B0E9D00000000000000000000000000000000000000000000000000000000000000000000000000000000000080E7C3
:2B0EC800000000000000000000000000000000000000000000000000000000000000000000000000000000000080E798
:2B0EF300000000000000000000000000000000000000000000000000000000000000000000000000000000000080E76D
:2B0F1E00020000000000000000000000000000000000000000000000000000000000000000000000000000000008EDB1
:2B0F4900000000000000000000000000000000000000000000000000000000000000000000000000000000000080E716
:2B0F7400000000000000000000000000000000000000000000000000000000000000000000000000000000000080E7EB
:2B0F9F00000000000000000000000000000000000000000000000000000000000000000000000000000000000080E7C0
:2B0FCA00000000000000000000000000000000000000000000000000000000000000000000000000000000000080E795
:2B0FF500000000000000000000000000000000000000000000000000000000000000000000000000000000000080E76A
:2B102000800008800008800008800008800008800008000000000020000220000220000220000220000220000280E742
:2B104B00800008800008800008800008800008800008000000000020000220000220000220000220000220000280E717
:2B107600000000000000000000000000000000000000000000000000000000000000000000000000000000000080E7E8
:2B10A100000000000000000000000000000000000000000000000000000000000000000000000000004000000080E381
:2B10CC00000000000000000000000000000000000000000000000000000000000000000000000000000000000080E792
:2B10F700000000000000000000000000000000000000000000000000020000000000000000000000000000000080E567
:2B112200000000000000000000000000000000000000000000000000020000000000000000000000004000000080E1FF
:2B114D00000000000000000000000000000000000000000000000000000000000000000000000000000000000080E710
:2B117800000000000000000000000000000000000000000000000000000000000000000000000000000000000080E7E5
:2B11A300000000000000000000000000000000000000000000000000000000000000000000000000000000000080E7BA
:2B11CE00000000000000000000000000000000000000000000000000000000000000000000000000000000000080E78F
:2B11F900080000000000000000000000000000000000000000000000000000000000000000000000000000000080EF54
:2B1224000000000000000000000000000000000000000000000000000000000000000000000000000000000000A0C53A
:2B124F00000000000000000000000000000000000000000000000000000000000000000000000000000000000080E70D
:2B127A00000000000000000000000000000000000000000000000000000000000000000000000000000000000080E7E2
:2B12A500080000000000000000000000000000000000000000000000000000000000000000000000000000000080EFA7
:2B12D000000000000000000000000000000000000000000000000000000000000000000000000000000000000080E78C
:2B12FB00000000000000000000000000000000000000000000000000000000000000000000000000000000000080E761
:2B132600000000000000000000000000000000000000000000000000000000000000000000000000000000000080E735
:2B135100000000000000000000000000000000000000000000000000000000000000000000000000000000000080E70A
:2B137C00000000000000000000000000000000000000000000000000000000000000000000000000000000000080E7DF
:2B13A700000000000000000000000000000000000000000000000000000000000000000000000000000000000090F695
:2B13D200000000000000000000000000000000000000000000000000000000000000000000000000000000000080E789
:2B13FD00000000000000000000000000000088000000000000000000000000000000000000000000000000000080EFCE
:2B142800000000000000000000000800000000000000000000000000000000000000000000000000000000002000E58C
:2B145300000000000000000000000000000000000000000000000000000000000000000000000000000000000080E707
:2B147E00080000000000000000000000000000000000000000000000000800000000000000000000000000000880EFBC
:2B14A900000000000000000000000000000000000000000000000000000000000000000000000000000000000080E7B1
:2B14D4000000000000000000000000000000000000000000000000000000000000000000000000000000000000C0A38A
:2B14FF00020000000000000000000000000000000000000000000000000000000000000000000000000000000080E55B
:2B152A000000000000000000000004000000000000000000000000000000000000000000000000000000000000C0E7EB
:2B155500000000000000000000000000000000000000000000000000011000010000010000000000011000001080E6D1
:2B158000000000000000000000000000000000000000000000000020000000000000000000000020004000000080E35D
:2B15AB00000000000000000000000200000000000000000000000000000000000000000000000000000000000080C5CE
:2B15D600000000000000000000000300000000000000000000000000000000000000000000000000000000000080D493
:2B160100000000000000000000008200200C4010000000000000000008020A000000000000000000040800000100EAB5
:2B162C00020000000000000000000000000000000000000000000000000000000000000000000020008200000008E502
:2B165700000000000000000000000000000000000000000000000000000000000000000000000000000000000408ABB1
:2B168200000000000000000000000000000000000000000000000000000000000000000000000000000000000090F6B7
:2B16AD00000000000000000000008200A02D4010000000000000000000000A000000000000000000048A00000108F9D9
:2B16D800000000000000000000000000000000000000000000000000000000000000000000000000000000000008EFF0
:2B170300020000000000000000000000000000000000000000000000000000000000000000000000000000000008EDC4
:2B172E00800008800008800008800008800008800008000000000020000220000220000220000220000220000280E72D
:2B175900800008800008800008800008800008800008000000000020000220000220000220000220000220000280E702
:2B1784000000000000000000000004000000100000000000000000400080400000200000000000000400000000809CE6
:2B17AF0002000000000000000060000000001E1000000000000000D88801B84000D8400000000098808900000008C69F
:2B17DA00020000000000000000000000000038000000000000000048822640000020000000000068820000000000FE72
:2B18050004000000000000000040080000001C000000000000000050000FB00400D00200000000F0002900000000DC76
:2B183000020000000000000000000200000018000000000000000008801000000000010000000008810000000000DF70
:2B185B00020000000000000000800000000038010000000000000068820680020080000000000068800000000080B19C
:2B188600020000000000000000802000000018000000000000000060000040010060000000000000000600000008DD91
:2B18B1000000000000000000008000000000380400000000000000604006400000E0010000000060000600000000B370
:2B18DC00000000000000000000000400000038000000000000000000040000000000000000000000044400000000D881
:2B19070000000000000000000060020000001E0000000000000000F88089180100980400000000F8800B00808980E291
:2B19320002000000000000000020000000001A000000000000000008820000000060000000000088000400800008D47C
:2B195D0000000000000000000040000000003C0400000000000000F00029100200F00100000000F0004B000029888255
:2B198800000000000000000000A00100000002000000000000000008800000000000010000000008000002800010CEA0
:2B19B300000000000000000000A001000000020000000000000000888200000000600000000000880208008000089052
:2B19DE00000000000000000000800100000018000000000000000060000660000000000000000060002400000608CF1E
:2B1A0900020000000000000000800100000018000000000000000060000660000060000000000060000C00000688A94E
:2B1A3400000000000000000000000000000000000000000000000000000040000000000000000000040001008080BF83
:2B1A5F00000000000000000000600A000000061000000000000000988489B84000980400000000F8800700800100A6FD
:2B1A8A000000000000000000000020000000800000000000000000408820400000000000000000088820008026008192
:2B1AB500020000000000000000C002000000340000000000000000500001B0040090400000000070000F00000708A10A
:2B1AE000020000000000000000004000000040000000000000000000800000000000000000000008822000801080A47B
:2B1B0B00040000000000000000000200000020000000000000000000C00000010000000000000008800000800E00C4EE
:2B1B3600020000000000000000001000000000000000000000000000020640000060000000000060000600000080A242
:2B1B61000200000000000000000000000000600000000000000000E0000640020060000000000060000600000600C53E
:2B1B8C00020000000000000000000000000000000000000000000020088000000060000000000000044400008008E56F
:2B1BB7000000000000000000006020000000260100000000000000588001980800980400000000F8800B00800100D370
:2B1BE20000000000000000000080010000001A000000000000000040A00608020000000000000008000400800680E556
:2B1C0D00000000000000000000C0010100003C0400000000000000500027100000F04000000000F0204B00002700C2AF
:2B1C380002000000000000000000000000001A000000000000000000800008000060010000000008000800800008B331
:2B1C630000000000000000000000000000001A000000000000000080811E08000080000000000008020000801608D518
:2B1C8E00000000000000000000000000000018000000000000000000020060000000000000000060001400000010A885
:2B1CB900000000000000000000000000000018000000000000000080000660000000000000000060000C00000688B256
:2B1CE400000000000000000000802100000008000000000000000020080000000000000000000000000001008008CEAD
:2B1D0F00020000000000000000600200000006100000000000000058808998080098080000000098880700800188E47A
:2B1D3A000000000000000000000000000000280000000000000000208010080200080100000000088100008016008BE9
:2B1D6500000000000000000000400A0000000C0000000000000000500101900000100000000000100047000007009D10
:2B1D9000000000000000000000004000000018000000000000000000A00008000008000000000008801000800000DB2D
:2B1DBB00020000000000000000000200000038010000000000000000800008000008000000000008800000802E089161
:2B1DE600020000000000000000000000000018000000000000000060000660000060000000000060000600000000FC30
:2B1E11000400000000000000000000000000380400000000000000E0010660000060000000000060000600000680BB18
:2B1E3C00020000000000000000800500000098000000000000000000008000000000000000000000040001000000BD1A
:2B1E6700020000000000000000E0010000003E000000000000000098840198080098080000000098800700808980B476
:2B1E920002000000000000000080010000001A000000000000000060800608000008000000000068801000800008AA68
:2B1EBD00000000000000000000C0090000005C0000000000000000F0011790400010010000000070010F00001180F3E8
:2B1EE800000000000000000000800200000002000000000000000000810028000008000000000008810000800000CFC2
:2B1F13000000000000000000008000000000020000000000000000E0802EA80400080000000000E88010008000008C5B
:2B1F3E0002000000000000000000200000001800000000000000000000000000006000000000000000060000068890BA
:2B1F6900000000000000000000800000000018000000000000000060000640010060000000000060000600000608BB7F
:2B1F94000000000000000000000004000000180000000000000000600080000000400000000000000000000000108155
:2B1FBF0000000000000000000060000000001E1000000000000000F88801180100D8080000000098888900808988D4E1
:2B1FEA000000000000000000000000000000380000000000000000688116000000480200000000088100008010889218
:2B2015000200000000000000004020000000140000000000000000F0000F10020050000000000090002100000908AB5C
:2B204000000000000000000000000200000018000000000000000008802000010008000000000008800000800000DFC3
:2B206B00000000000000000000000000000038010000000000000008800600000068020000000008800000800000DF32
:2B209600000000000000000000802000000018000000000000000060000000000040000000000060000600000680B02B
:2B20C100020000000000000000000000000038040000000000000060000660000060010000000060000600000688B5E6
:2B20EC00000000000000000000002100000010000000000000000000000000000000000000000000040000008080E9AB
:2B21170000000000000000000060030000001E1000000000000000F88889180100F80800000000F8804100800780C961
:2B214200000000000000000000000100000030000000000000000008810000000008020000000008400E00800081F85F
:2B216D00000000000000000000400B000000140000000000000000700019100200F00000000000F0000F00000F80B11E
:2B2198000200000000000000000041000000000000000000000000088100000100080100000000080006008000889799
:2B21C3000000000000000000008003000000200100000000000000888000000000080000000000880106008018009185
:2B21EE00000000000000000000000100000000000000000000000060000600040060000000000060000600000680F21D
:2B2219000000000000000000000007000000200400000000000000600006C0000060000000000060000600000600F28B
:2B224400000000000000000000000000000000000000000000000000000000000000000000000000000000000080E708
:2B226F00000000000000000000800000000008000000000000000020000220000020000000000020000200000280C5F1
:2B229A00800008800008800008000008800000800008000000000000000000000200000220000200000020000080C5E6
:2B22C500800008800008800008800008800008800008000000000020000220000220000220000220000220000280E78B
:2B22F000000000000000000000000E0000054011000000000000004808000822A0880000000000C0940C00000082D10A
:2B231B00000000000000000000000000000000000000000000000040000000000000000000000000100000000080B314
:2B234600000000000000000000000000000000000000000000000000000000000000000000000000000000000080E705
:2B237100000000000000000000800000000000000000000000000000000000000000000000000000008000000000E75A
:2B239C00000000000000000000000E00000440110000000000000048080008222088000000000080940800000282EA07
:2B23C700000000000000000000400001000000000000000000000000000000000000000000000000000000000080B773
:2B23F200000000000000000000000000000000000000000000000000000000000000000000000010000100000080E748
:2B241D00000000000000000000000000000000000000000000000000000000000000000000000000000000000080E72D
:2B244800000000000000000000000000000000000000000000000080000000000000000000000000000200000000C522
:2B2473000000000000000000000000000000041000000000000000000000000000000000000000001004000000D0B690
:2B249E00000000000000000000000000000000000000000000000000080020000000000000000080200001000000FD4D
:2B24C900080000000000000000000000000000000000000000000000000020200000200000000000000200000080EF0F
:2B24F400000000000000000000000000000000000000000000000000000000000000000000000000000000000080E756
:2B251F00000000000000000000000000000000000000000000000020400000000020000000000000000000000080A7EA
:2B254A000000000000000000000000000000000000000000000000000000000000000000000000000000000000C0A303
:2B257500000000000000000000000000000000000000000000000000000000000000000000000000000100000080F6C4
:2B25A000000000000000000000000000000000000000000000000000000000000000000000000000000000000080E7A9
:2B25CB00000000000000000000000000000000000000000000000000000000000000000000000000000000000090F65F
:2B25F600000000000000000000000000000000000000000000000000000000000000000000000000000000000080E753
:2B262100000000000000000000000000000000000000000000000000000000000000000000000000000000000080E727
:2B264C00000000000000000000000000000000000000000000000000000000000000000000000000000000000080E7FC
:2B267700000000000000000000000000000000000000000000000000000000000000000000000000000000000080E7D1
:2B26A200000000000000000000000000000000000000000000000000000000000000000000000000000000000080E7A6
:2B26CD00000000000000000000000000000000000000000000000000000000000000000000000000000000000008EFEB
:2B26F800000000000000000000000000000000000000000000000000000000000000000000000000000000000080E750
:2B272300000000000000000000000000000000000000000000000000000000000000000000000000000000000080E724
:2B274E00000000000000000000000000000000000000000000000000000000000000000000000000000000000080E7F9
:2B277900000000000000000000000000000000000000000000000000000000000000000000000000000000000080E7CE
:2B27A400000000000000000000000000000000000000000000000000000000000000000000000000000000000008EF13
:2B27CF00000000000000000000000000000000000000000000000000000000000000000000000000000000000080E778
:2B27FA00000000000000000000000000000000000000000000000000000000000000000000000000000000000080E74D
:2B282500000000000000000000000000000000000000000000000000000000000000000000000000000000000080E721
:2B285000000000000000000000000000000000000000000000000000000000000000000000000000000000000080E7F6
:2B287B00000000000000000000000000000000000000000000000000000000000000000000000008000000000000EF3B
:2B28A600020000000000000000000000000000000000000000000000000000000000000000000000000000000008ED10
:2B28D100000000000000000000000000000000000000000000000000000000000000000000000000000000000080E775
:2B28FC00000000000000000000000000000000000000000000000000000000000000000000000008000000000000EFBA
:2B292700000000000000000000000000000000000000000000000000000000000000000000000000000000000080E71E
:2B295200000000000000000000000000000000000000000000000000000000000000000000000000000000000080E7F3
:2B297D00020000000000000000000000000000000000000000000000000000000000000000000000000000000008ED38
:2B29A800800008800008800008800008800008800008000000000020000220000220000220000220000220000280E7A1
:2B29D300800008800008800008800008800008800008000000000020000220000220000220000220000220000280E776
:2B29FE00000000000000000000000000000000000000000000000000000000000000000000000000000000000080E747
:2B2A2900020000000000000000000000000000000000000000000000000000000000000000000000000000000008ED8B
:2B2A5400000000000000000000000000000000000000000000000000000000000000000000000000000000000080E7F0
:2B2A7F00000000000000000000000000000000000000000000000000000000000000000000000000000000000080E7C5
:2B2AAA00000000000000000000000000000000000000000000000000000000000000000000000000000000000080E79A
:2B2AD500000000000000000000000000000000000000000000000000000000000000000000000000000000000080E76F
:2B2B0000020000000000000000000000000000000000000000000000000000000000000000000000000000000008EDB3
:2B2B2B00000000000000000000000000000000000000000000000000000000000000000000000000000000000080E718
:2B2B5600000000000000000000000000000000000000000000000000000000000000000000000000000000000080E7ED
:2B2B8100000000000000000000000000000000000000000000000000000000000000000000000000000000000080E7C2
:2B2BAC00020000000000000000000000000000000000000000000000000000000000000000000000000000000008ED07
:2B2BD700000000000000000000000000000000000000000000000000000000000000000000000000000000000080E76C
:2B2C0200000000000000000000000000000000000000000000000000000000000000000000000000000000000080E740
:2B2C2D00000000000000000000000000000000000000000000000000000000000000000000000000000000000080E715
:2B2C5800000000000000000000000000000000000000000000000000000000000000000000000000000000000080E7EA
:2B2C8300020000000000000000000000000000000000000000000000000000000000000000000000000000000008ED2F
:2B2CAE00000000000000000000000000000000000000000000000000000000000000000000000000000000000080E794
:2B2CD900000000000000000000000000000000000000000000000000000000000000000000000000000000000080E769
:2B2D0400000000000000000000000000000000000000000000000000000000000000000000000000000000000080E73D
:2B2D2F00020000000000000000000000000000000000000000000000000000000000000000000000000000000008ED82
:2B2D5A00000000000000000000000000000000000000000000000000000000000000000000000000000000000008EF57
:2B2D8500000000000000000000000000000000000000000000000000000000000000000000000000000000000090F69D
:2B2DB000000000000000000000000000000000000000000000000000000000000000000000000000000000000008EF01
:2B2DDB00000000000000000000000000000000000000000000000000000000000000000000000000000000000008EFD6
:2B2E0600020000000000000000000000000000000000000000000000000000000000000000000000000000000008EDAA
:2B2E3100000000000000000000000000000000000000000000000000000000000000000000000000000000000080E70F
:2B2E5C00000000000000000000000000000000000000000000000000000000000000000000000000000000000080E7E4
:2B2E8700000000000000000000000000000000000000000000000000000000000000000000000000000000000080E7B9
:2B2EB200020000000000000000000000000000000000000000000000000000000000000000000000000000000008EDFE
:2B2EDD00000000000000000000000000000000000000000000000000000000000000000000000000000000000080E763
:2B2F0800000000000000000000000000000000000000000000000000000000000000000000000000000000000080E737
:2B2F3300000000000000000000000000000000000000000000000000000000000000000000000000000000000080E70C
:2B2F5E00000000000000000000000000000000000000000000000000000000000000000000000000000000000080E7E1
:2B2F8900020000000000000000000000000000000000000000000000000000000000000000000000000000000008ED26
:2B2FB400000000000000000000000000000000000000000000000000000000000000000000000000000000000080E78B
:2B2FDF00000000000000000000000000000000000000000000000000000000000000000000000000000000000080E760
:2B300A00000000000000000000000000000000000000000000000000000000000000000000000000000000000080E734
:2B303500020000000000000000000000000000000000000000000000000000000000000000000000000000000008ED79
:2B306000000000000000000000000000000000000000000000000000000000000000000000000000000000000080E7DE
:2B308B00000000000000000000000000000000000000000000000000000000000000000000000000000000000080E7B3
:2B30B600000000000000000000000000000000000000000000000000000000000000000000000000000000000080E788
:2B30E100000000000000000000000000000000000000000000000000000000000000000000000000000000000080E75D
:2B310C00020000000000000000000000000000000000000000000000000000000000000000000000000000000008EDA1
:2B313700000000000000000000000000000000000000000000000000000000000000000000000000000000000080E706
:2B316200000000000000000000000000000000000000000000000000000000000000000000000000000000000080E7DB
:2B318D00000000000000000000000000000000000000000000000000000000000000000000000000000000000080E7B0
:2B31B800020000000000000000000000000000000000000000000000000000000000000000000000000000000008EDF5
:2B31E300000000000000000000000000000000000000000000000000000000000000000000000000000000000080E75A
:2B320E00000000000000000000000000000000000000000000000000000000000000000000000000000000000080E72E
:2B323900000000000000000000000000000000000000000000000000000000000000000000000000000000000080E703
:2B326400000000000000000000000000000000000000000000000000000000000000000000000000000000000080E7D8
:2B328F00020000000000000000000000000000000000000000000000000000000000000000000000000000000008ED1D
:2B32BA00000000000000000000000000000000000000000000000000000000000000000000000000000000000080E782
:2B32E500000000000000000000000000000000000000000000000000000000000000000000000000000000000080E757
:2B331000000000000000000000000000000000000000000000000000000000000000000000000000000000000080E72B
:2B333B00020000000000000000000000000000000000000000000000000000000000000000000000000000000008ED70
:2B336600000000000000000000000000000000000000000000000000000000000000000000000000000000000080E7D5
:2B339100000000000000000000000000000000000000000000000000000000000000000000000000000000000080E7AA
:2B33BC00000000000000000000000000000000000000000000000000000000000000000000000000000000000080E77F
:2B33E700000000000000000000000000000000000000000000000000000000000000000000000000000000000080E754
:2B341200020000000000000000000000000000000000000000000000000000000000000000000000000000000008ED98
:2B343D00000000000000000000000000000000000000000000000000000000000000000000000000000000000080E7FD
:2B346800000000000000000000000000000000000000000000000000000000000000000000000000000000000080E7D2
:2B349300000000000000000000000000000000000000000000000000000000000000000000000000000000000080E7A7
:2B34BE00000000000000000000000000000000000000000000000000000000000000000000000000000000000080E77C
:2B34E900000000000000000000000000000000000000000000000000000000000000000000000000000000000080E751
:2B351400800008800008800008800008800008800008000000000020000220000220000220000220000220000280E729
:2B353F00800008800008800008800008800008800008000000000020000220000220000220000220000220000280E7FE
:2B356A00000000000000000000000000000000000000000000000000000000000000000000000000000000000080E7CF
:2B359500000000000000000000000000000000000000000000000000000000000000000000000000000000000080E7A4
:2B35C000000000000000000000000000000000000000000000000000000000000000000000000000000000000080E779
:2B35EB00000000000000000000000000000000000000000000000000000000000000000000000000000000000080E74E
:2B361600000000000000000000000000000000000000000000000000000000000000000000000000000000000080E722
:2B364100000000000000000000000000000000000000000000000000000000000000000000000000000000000080E7F7
:2B366C00000000000000000000000000000000000000000000000000000000000000000000000000000000000080E7CC
:2B369700000000000000000000000000000000000000000000000000000000000000000000000000000000000080E7A1
:2B36C200000000000000000000000000000000000000000000000000000000000000000000000000000000000080E776
:2B36ED00000000000000000000000000000000000000000000000000000000000000000000000000000000000080E74B
:2B371800000000000000000000000000000000000000000000000000000000000000000000000000000000000080E71F
:2B374300000000000000000000000000000000000000000000000000000000000000000000000000000000000080E7F4
:2B376E00000000000000000000000000000000000000000000000000000000000000000000000000000000000080E7C9
:2B379900000000000000000000000000000000000000000000000000000000000000000000000000000000000080E79E
:2B37C400000000000000000000000000000000000000000000000000000000000000000000000000000000000080E773
:2B37EF00000000000000000000000000000000000000000000000000000000000000000000000000000000000080E748
:2B381A00000000000000000000000000000000000000000000000000000000000000000000000000000000000080E71C
:2B384500000000000000000000000000000000000000000000000000000000000000000000000000000000000080E7F1
:2B387000000000000000000000000000000000000000000000000000000000000000000000000000000000000080E7C6
:2B389B00000000000000000000000000000000000000000000000008010000000000000000000008400100800C80FBA9
:2B38C600000000000000000000000000000000000000000000000020000000000000000000000020008201008280F71B
:2B38F100000000000000000000000000000000000000000000000000000000000000000000000000000000000080E745
:2B391C00000000000000000000000000000000000000000000000000000000000000000000000000000000000080E719
:2B39470040100441100441100441100441100441100401000000003804411004411004411004413884E31084E380E75E
:2B397200601886611886611886611886611886611886010000000058866118866118866118866158866519866581E745
:02399D00FFFF2A
:00000001FF
